:1000000000308A00CD2800000030A1001F08C3394D
:1000100021049F000D30A000A00B0C289F149F18F6
:100020000F2883161E088312A5001E08A6000430A0
:10003000A1001F08C33921049F000D30A000A00BB0
:100040001F289F149F18222883161E088312A700BA
:100050001E08A8000830A1001F08C33921049F0012
:100060000D30A000A00B32289F149F18352883164E
:100070001E088312AB001E08AC000C30A1001F0844
:10008000C33921049F000D30A000A00B45289F1408
:100090009F18482883161E088312A9001E08AA006C
:1000A000F028A101A201A001A3013608031D5B28CD
:1000B0003508031975281030B7000310B30DB40DBF
:1000C000A00DA30D36082302031D68283508200261
:1000D000031C71283508A002031CA3033608A302E1
:1000E0000314A10DA20DB70B5D2800009F28B201DB
:1000F000B101B208031D91283108123C031C91285C
:1001000085160830A000A00B83280000851203305C
:10011000A000A00B892800000000B10A0319B20A50
:1001200079288512D830A000A00B942800002F0851
:10013000B4002E08B300B6010A30B50051282208D9
:10014000AF002108AE00B201B10132082F02031C3A
:10015000B928031DAF282E0831020318B928013031
:10016000B0000000000000000000B10A0319B20A4C
:10017000A52800342E30840000080319CC28023052
:10018000A100A001A00BC228A10BC1289730A0009C
:10019000A00BC828800BBF280C2984011F308305C1
:1001A0001F1383161F149F141F159F1507308312EA
:1001B0009F00703083168F001F30650083121F135D
:1001C00083161F149F141F159F151F129F161F13B0
:1001D00083129F171F14703083168F008312042818
:1001E00085122808AF002708AE0077202A08AF0044
:1001F0002908AE0077202608AF002508AE0077203A
:100200002C08AF002B08AE0077200230AF00AE0103
:0E02100077200A30AE00BA288316EE2863006D
:02400E00C43FAD
:00000001FF
